:100000000C9464000C948C000C948C000C948C0068
:100010000C949A000C948C000C948C000C948C0022
:100020000C948C000C948C000C948C000C940B0B96
:100030000C948C000C948C000C948C000C948C0010
:100040000C94DC0B0C948C000C941C0E0C946A0E1B
:100050000C948C000C948C000C948C000C948C00F0
:100060000C948C000C948C000000000024002700ED
:100070002A0000000000250028002B0000000000DE
:1000800023002600290004040404040404040202DA
:100090000202020203030303030301020408102007
:1000A0004080010204081020010204081020000012
:1000B0000007000201000003040600000000000029
:1000C00000008E004407D60F11241FBECFEFD8E0EA
:1000D000DEBFCDBF11E0A0E0B1E0E8EAFAE202C085
:1000E00005900D92A838B107D9F713E0A8E8B1E060
:1000F00001C01D92A337B107E1F710E0C8ECD0E0D2
:1001000004C02297FE010E944E15C23CD107C9F7D8
:100110000E940C0E0C9452150C94000088E891E09B
:100120000E949709089581E593E060E071E00E94E4
:100130008B1208951F920F920FB60F921124EF9217
:10014000FF920F931F932F933F934F935F936F9360
:100150007F938F939F93AF93BF93EF93FF93809180
:100160006502882309F445C08EE00E94B90D892BF1
:1001700021F481E0809362023CC080916202882376
:10018000C1F1109262028091630290916402019623
:1001900090936402809363020E94240C0E94A01337
:1001A00020E030E040E85CE30E9456140E947413A3
:1001B0009B01AC018091660290916702A091680258
:1001C000B091690279018A01E81AF90A0A0B1B0B3E
:1001D000D801C7014A97A105B10518F081E08093C5
:1001E0006A0220936602309367024093680250933C
:1001F0006902FF91EF91BF91AF919F918F917F9194
:100200006F915F914F913F912F911F910F91FF90AF
:10021000EF900F900FBE0F901F90189583E060E055
:1002200070E00E94C60C8BE060E070E00E94C60C9B
:1002300080917601882399F480918B0190918C01B3
:10024000A0918D01B0918E0180936E0290936F0208
:10025000A0937002B093710281E080936D020895C3
:10026000AF92BF92CF92DF92EF92FF920F931F93C4
:10027000CF93DF93C0916B02D0916C02CE010197B6
:10028000029758F00F2EF0E0AF2EF0E0BF2EF0E016
:10029000CF2EF0E0DF2EF02D18C060916302709138
:1002A0006402882777FD8095982F0E94A21320E092
:1002B00030E044E353E40E9407135B016C01229792
:1002C00021F4D7FAD094D7F8D09410926402109207
:1002D0006302E090DA01F090DB010091DC01109103
:1002E000DD0180E090E0A0E0B0E08093DA0190933F
:1002F000DB01A093DC01B093DD0181E593E060E1D7
:1003000071E00E94A11181E593E0B601A50122E010
:1003100030E00E94881281E593E068E171E00E947C
:10032000A11181E593E0B801A70122E030E00E942D
:10033000881281E593E06AE171E00E948B12DF91FF
:10034000CF911F910F91FF90EF90DF90CF90BF90D2
:10035000AF9008950E94300181E593E06CE171E077
:100360000E948B1210926D0281E0809376011092B0
:100370006C0210926B0280918B0190918C01A09184
:100380008D01B0918E018093DE019093DF01A093E7
:10039000E001B093E1010895CF92DF92EF92FF92D6
:1003A0000F931F93DF93CF93CDB7DEB7CE57D040D7
:1003B0000FB6F894DEBF0FBECDBF8E010F5F1F4F8B
:1003C00078018FE7C82ED12CCC0EDD1E87E792E096
:1003D00068E570E04EE350E021E030E00E9454090F
:1003E00087E792E00E943007D7018D937D01AC151D
:1003F000BD0561F7E4EEF1E0D8013C9120E01196F3
:100400008C9190E0822B932B819391930E5F1F4FE1
:100410000E151F0589F7C258DF4F0FB6F894DEBFDF
:100420000FBECDBFCF91DF911F910F91FF90EF9045
:10043000DF90CF9008950F931F9307E712E0C80154
:1004400068E570E04DE350E021E030E00E9454099F
:10045000C8010E94300790E09695879596958795FC
:1004600081701F910F9108951F9387E792E068E5CF
:1004700070E042E250E021E030E00E94540987E75A
:1004800092E00E943007882381F387E792E068E5D5
:1004900070E047E250E022E030E00E94540987E734
:1004A00092E00E943007182F87E792E00E94300701
:1004B000512F40E0282F30E0242B352BC9011F910C
:1004C000089585E060E070E00E94C60C86E060E080
:1004D00070E00E94C60C83E060E070E00E94C60CF1
:1004E0008BE060E070E00E94C60C88E891E00E941A
:1004F000B10908951F93CF93DF9380919701909155
:1005000098018137910571F46091990170919A0178
:1005100085E00E94C60C8CE060E00E94650D89E0D9
:1005200061E010C08F36910581F46091990170915E
:100530009A0185E00E94C60C8CE061E00E94650D86
:1005400089E060E00E94650DCDC18037910541F4DE
:100550006091990170919A0186E00E94C60CC2C117
:100560008637910579F488E891E06AE070E00E94AE
:10057000040B6091990170919A0188E891E00E94C2
:100580001D0AB0C18737910529F488E891E00E94DF
:10059000B109A8C18D36910549F48FEB92E060E076
:1005A00070E0409199010E94D00B9CC18636910564
:1005B00081F08236910569F08C36910551F08237D1
:1005C000910539F08A37910521F08536910509F0BA
:1005D000D8C06091990170919A0183E00E94C60C85
:1005E00060919B0170919C018BE00E94C60C8091F0
:1005F00097019091980186369105B9F482E061E007
:100600000E94650D84E060E00E94650D87E060E077
:100610000E94650D88E061E00E94650D10926D02F8
:100620001092760181E090E019C082369105D9F4EC
:1006300082E060E00E94650D84E061E00E94650D4B
:1006400087E061E00E94650D88E060E00E94650D32
:1006500010926D021092760182E090E090936C020D
:1006600080936B023FC18C369105B9F482E060E063
:100670000E94650D84E061E00E94650D87E060E006
:100680000E94650D88E061E00E94650D10926D0288
:100690001092760183E090E0E1CF82379105B9F4C2
:1006A00082E061E00E94650D84E060E00E94650DDB
:1006B00087E061E00E94650D88E060E00E94650DC2
:1006C00010926D021092760184E090E0C7CF8A37D5
:1006D0009105B9F482E060E00E94650D84E061E07C
:1006E0000E94650D87E060E00E94650D88E061E092
:1006F0000E94650D10926D021092760183E090E0E9
:100700001AC08536910509F0EDC082E061E00E94D3
:10071000650D84E060E00E94650D87E061E00E9465
:10072000650D88E060E00E94650D10926D021092E8
:10073000760184E090E090936C0280936B0290913C
:100740009D0180E020919F013091A001822B932B8D
:10075000AA2797FDA095BA2F20918B0130918C018B
:1007600040918D0150918E01820F931FA41FB51FE0
:100770008093930190939401A0939501B093960177
:10078000B1C08337910519F40E940E01ABC08836C1
:10079000910549F582E060E00E94650D84E060E02B
:1007A0000E94650D87E060E00E94650D88E060E0D2
:1007B0000E94650D80917601882309F093C0809195
:1007C0008B0190918C01A0918D01B0918E0180934D
:1007D0006E0290936F02A0937002B093710281E059
:1007E00080936D027FC08837910529F481E593E0FD
:1007F00063E271E075C08937910519F40E94930096
:1008000071C08336910529F481E593E06EE271E0D1
:1008100067C08936910511F5109262021092640248
:100820001092630221E0209365022093D90180E0B9
:1008300090E0A0E0B0E08093DA019093DB01A09318
:10084000DC01B093DD0110926A0210926D022093D8
:10085000760110926C0210926B0244C08A369105A8
:1008600049F40E94300110926502109262021092C7
:10087000D90138C08B36910519F40E94300132C07D
:100880008833910591F4C0E0D0E08FEB92E0BE0197
:1008900040E00E94D00B219682E0C030D807A9F733
:1008A00081E593E06FE271E01BC0C997D9F48FEB4B
:1008B00092E060E070E00E94C90B182F81E593E0A0
:1008C0006FE371E00E94A11181E593E0612F70E078
:1008D0004AE050E00E948E1181E593E06AE171E008
:1008E0000E948B12DF91CF911F91089581E593E0D3
:1008F0000E945D0F9C018D30910519F08A309105A1
:1009000071F48091D7019091D80118161906BCF4A2
:100910000E947A021092D8011092D7010895809116
:10092000D7019091D801FC01EE0FFF1FE956FE4F51
:100930003183208301969093D8018093D701089545
:100940008F929F92AF92BF92CF92DF92EF92FF92DF
:100950000F931F93CF93DF930E94240C0E94A01348
:1009600020E030E040E85CE30E9456140E947413DB
:1009700060938B0170938C0180938D0190938E0115
:100980008091D901882309F487C08091760188235A
:1009900009F082C00E941B02882309F47DC00E94D6
:1009A000CC0180916D02882321F180916B0290919E
:1009B0006C0203970297E8F4BB2480918B0190911D
:1009C0008C01A0918D01B0918E0120918F01309109
:1009D00090014091910150919201821B930BA40BC5
:1009E000B50B81359105A105B10520F0BB24B39469
:1009F00001C0BB248090E2019090E301C090DA0135
:100A0000D090DB01E090DC01F090DD01C4EED1E09C
:100A1000AA2408811981080D191DB801882777FDBE
:100A20008095982F0E94A21320E030E04AE753E41B
:100A30000E94561420E03EEF4FEF56EC0E94071341
:100A40009B01AC010E949F1220E030E04AE754E491
:100A50000E9407139B01AC01C701B6010E949F12BF
:100A60006B017C01BB2039F00B561F4F0B5211401C
:100A700010F4AA24A394229682E0C236D80749F63D
:100A8000C092DA01D092DB01E092DC01F092DD014C
:100A9000AA2011F00E94AA01E0908B01F0908C0135
:100AA00000918D0110918E01A8019701205D3740C2
:100AB000404050408091DE019091DF01A091E00123
:100AC000B091E10182179307A407B50740F580EDC7
:100AD000E81687E0F80680E0080780E01807F8F0DD
:100AE00080917601882359F00E9434020E943402DA
:100AF000909581959F4F9093E3018093E2018091BF
:100B00008B0190918C01A0918D01B0918E01809309
:100B1000DE019093DF01A093E001B093E1018091A9
:100B20006D02882349F180918B0190918C01A091F5
:100B30008D01B0918E01885E9340A040B04020911D
:100B40006E0230916F02409170025091710228172D
:100B500039074A075B0780F48091D901882361F047
:100B600080916502882341F081E593E06FE471E0B4
:100B70000E948B120E94AA0180916A02882399F038
:100B800010926A0280916502882369F080916D025B
:100B9000882349F080916B0290916C020197029733
:100BA00010F40E94AA012091930130919401409188
:100BB0009501509196012115310541055105B9F076
:100BC00080918B0190918C01A0918D01B0918E014B
:100BD000281739074A075B0750F40E940E0110924C
:100BE000930110929401109295011092960181E563
:100BF00093E00E942C0F20918B0130918C01409149
:100C00008D0150918E01181619065CF420938F0106
:100C10003093900140939101509392010E94760489
:100C200023C0205137424040504080918F01909125
:100C30009001A0919101B091920182179307A407AE
:100C4000B50790F40E94610280918B0190918C0114
:100C5000A0918D01B0918E0180938F0190939001AE
:100C6000A0939101B0939201DF91CF911F910F91C9
:100C7000FF90EF90DF90CF90BF90AF909F908F90BC
:100C80000895CF93DF938FEB92E060E070E00E94D5
:100C9000C90BC82FD0E0CE014E978734910548F09C
:100CA0008FEB92E060E070E046E40E94D00BC6E477
:100CB000D0E088E891E06AE070E00E94040B88E8E8
:100CC00091E0BE010E941D0A64EF71E080E090E0B7
:100CD0000E94320C88E891E00E94B10983E061E053
:100CE0000E94260D8BE061E00E94260D82E061E00B
:100CF0000E94260D84E061E00E94260D87E061E0FD
:100D00000E94260D88E061E00E94260D89E061E0E6
:100D10000E94260D86E061E00E94260D8CE061E0D5
:100D20000E94260D8EE060E00E94260D8091B100A9
:100D300087608093B10085B5887F816085BD83E041
:100D400060E070E00E94C60C8BE060E070E00E9402
:100D5000C60C82E061E00E94650D84E060E00E94C4
:100D6000650D87E061E00E94650D88E060E00E940B
:100D7000650D87E792E00E94170787E792E061E040
:100D80000E94280787E792E068E570E040E050E0C5
:100D90002CEC30E00E94940987E792E068E570E06F
:100DA00041E050E020E230E00E94940987E792E0C1
:100DB00068E570E042E050E023E130E00E949409F1
:100DC00087E792E068E570E043E150E020E230E040
:100DD0000E94940987E792E068E570E048E150E0FE
:100DE00024E530E00E94940987E792E068E570E02E
:100DF00047E150E02EE330E00E949409F89482E04D
:100E00008093680081E080936C00789481E593E0A2
:100E100040E052EC61E070E00E94A50E81E593E0B5
:100E200060E671E00E948B12DF91CF910895449AA1
:100E3000459AE9EBF0E080818E7F808380818D7F11
:100E4000808388E48093B80084E48093BC00089594
:100E5000662311F488E401C08CE08093B800089503
:100E6000FC018091720290917402981B909373021E
:100E7000882319F4109273020895815080937202AE
:100E8000E90FF11D828108950895EF92FF920F936B
:100E90001F930E94240C7B018C0184E98093BC0089
:100EA0001BC021153105E1F00E94240C6E197F0949
:100EB000800B910B209175023091760240E050E05A
:100EC000621773078407950738F01092BC0084E41A
:100ED0008093BC0081E009C02091750230917602B8
:100EE0008091BC0084FDDDCF80E01F910F91FF90C9
:100EF000EF900895CF92DF92EF92FF921F93162FFB
:100F00000E94240C6B017C01112311F084EC01C0C0
:100F100084E88093BC001BC021153105E1F00E94DC
:100F2000240C6C197D098E099F092091750230915E
:100F3000760240E050E0621773078407950738F0A7
:100F40001092BC0084E48093BC0091E019C0209111
:100F50007502309176028091BC0087FFDDCF8091D1
:100F6000B900887F883349F49091B900987F109236
:100F7000BC0084E48093BC0003C09091B900987FCA
:100F8000892F1F91FF90EF90DF90CF900895EF92FF
:100F9000FF920F931F93CF93DF93EC016093BB00FD
:100FA0000E94240C7B018C0184E88093BC001BC050
:100FB00021153105E1F00E94240C6E197F09800B88
:100FC000910B209175023091760240E050E062175B
:100FD00073078407950738F01092BC0084E480936F
:100FE000BC0011E020C02091750230917602809102
:100FF000BC0087FFDDCF8091B900887F883211F473
:1010000010E011C01091B900187F8091B900887F5D
:10101000803321F4CE010E94450705C01092BC0028
:1010200084E48093BC00812FDF91CF911F910F91B9
:10103000FF90EF900895EF92FF920F931F93CF933D
:10104000DF93EC016093BB000E94240C7B018C01B8
:1010500084E88093BC001BC021153105E1F00E949B
:10106000240C6E197F09800B910B20917502309131
:10107000760240E050E0621773078407950738F066
:101080001092BC0084E48093BC0011E01DC020914C
:101090007502309176028091BC0087FFDDCF809190
:1010A000B900887F883179F08091B900887F8034D9
:1010B00099F409C08091B900887F8834B1F4CE01D9
:1010C0000E94450701C010E0812FDF91CF911F9151
:1010D0000F91FF90EF9008951091B900187F8091C3
:1010E000B900887F803231F7EACF1092BC0084E4E7
:1010F0008093BC00E9CFEF92FF920F931F930E9461
:10110000240C7B018C0184EA8093BC001BC0211558
:101110003105E1F00E94240C6E197F09800B910BC0
:10112000209175023091760240E050E0621773071B
:101130008407950738F01092BC0084E48093BC00CB
:1011400091E021C020917502309176028091BC001F
:1011500087FFDDCF8091B900887F883099F080913A
:10116000B900887F8031A9F40DC09091B900987FB3
:101170001092BC0084E48093BC0005C09091B9003B
:10118000987F01C090E0892F1F910F91FF90EF9001
:1011900008958091B900887F883381F7E6CFEF9278
:1011A000FF920F931F93CF93DF93EC01162F042F21
:1011B000E22E1092720210927302222311F4EE2496
:1011C000E394EA94E982E3941882CE010E947B08BA
:1011D0008883882309F061C0110FCE01612F0E941E
:1011E0001B088883882329F0813009F056C082E0EB
:1011F00054C0CE01602F0E94C7078883882329F03E
:10120000813009F04AC083E048C0CE010E947B08CB
:101210008883882329F0813009F03FC084E03DC0F5
:101220001F5FCE01612F0E941B088883882319F459
:101230008E01FF2425C0813081F585E02EC0898193
:10124000F81651F4CE0160E00E947A07888381305D
:1012500019F1883551F021C0CE0161E00E947A0772
:1012600088838130C9F08035C1F48091BB00F801DA
:101270008283F394F0927202F09274020F5F1F4F18
:10128000FE14E8F2CE010E9445078883882329F0E6
:10129000813019F487E001C086E0DF91CF911F9182
:1012A0000F91FF90EF9008950E94CF080895FF924C
:1012B0000F931F93CF93DF93EC01162F042FF22E81
:1012C00018820E947B088883882341F5110FCE0184
:1012D000612F0E941B088883882321F08130F1F45C
:1012E00082E01CC0CE01602F0E94C707888388233C
:1012F00039F4CE016F2D0E94C7078883882319F027
:10130000813061F40AC0CE010E944507888388239A
:1013100029F0813019F487E001C083E0DF91CF919B
:101320001F910F91FF9008950E9457090895FC01A5
:10133000809199028C3090F480838F5F8093990222
:10134000815090E0FC01EE0FFF1FE80FF91FE656F9
:10135000FD4F88EB9BE09283818308958FEF80831C
:101360000895DC018C9190E0FC01EE0FFF1FE80F67
:10137000F91FE656FD4F80818F7B80838C916CE056
:101380000E94DC1490E0AC01440F551F480F591F18
:10139000440F551F440F551F20E030E0C901840F52
:1013A000951FFC01EE0FFF1FE80FF91FE656FD4FDA
:1013B000808186FD05C02F5F3F4F2C30310571F7CE
:1013C0000895FC0120812C30B8F58181992787FD93
:1013D000909548E850E0481B590B440F551F440FA7
:1013E000551F6417750784F08281992787FD9095B2
:1013F00048E552E0481B590B440F551F440F551F39
:10140000641775070CF4AB0142505040CA01AA277B
:1014100097FDA095BA2F880F991FAA1FBB1F4FB722
:10142000F89430E0F901EE0FFF1FE20FF31FE656CC
:10143000FD4F928381834FBF0895AF92BF92CF92A9
:10144000DF92EF92FF920F931F93CF93DF93EC0104
:101450009B0182E0603278070CF048C077FF03C040
:1014600020E030E005C0653B710514F024EB30E06E
:1014700000D000D0B901882777FD8095982F298169
:10148000332727FD3095E8E8AE2EB12CA21AB30A17
:10149000AA0CBB1CAA0CBB1CCC24B7FCC094DC2C33
:1014A000EA81FF27E7FDF09528E532E02E1B3F0B90
:1014B000220F331F220F331F442737FD4095542F2F
:1014C000EDB7FEB7218332834383548320E030E0BD
:1014D00040E050E004EBE02EF12C012D112D0E9494
:1014E0002C109B010F900F900F900F90CE01B9011F
:1014F0000E94E109DF91CF911F910F91FF90EF9032
:10150000DF90CF90BF90AF900895CF92DF92EF928F
:10151000FF921F93CF93DF93EC01162F7A0169019D
:1015200088818C3008F064C0862F61E00E94260D0F
:10153000888190E0FC01EE0FFF1FE80FF91FE656CF
:10154000FD4F1F738081807C812B808380E292E03D
:101550008E199F0964E070E00E94E814698380E6B8
:1015600099E08C199D0964E070E00E94E8146A8398
:10157000A8818A2F6CE00E94DC14682F70E0AB0118
:10158000440F551F460F571F440F551F440F551F3B
:1015900020E030E0C901840F951FFC01EE0FFF1F12
:1015A000E80FF91FE656FD4F808186FD15C02F5FBD
:1015B0003F4F2C30310571F724C01092800082E03B
:1015C000809381001092850010928400B19A8091DE
:1015D0006F00826080936F008A2F90E0FC01EE0F15
:1015E000FF1FE80FF91FE656FD4F8081806480835E
:1015F0008881DF91CF911F91FF90EF90DF90CF9086
:101600000895672BD1F2E8CF40E252E020E639E0BE
:101610000E94850A08951F920F920FB60F9211240F
:101620002F933F934F935F936F937F938F939F93EA
:10163000AF93BF93EF93FF938091BE0287FF05C0E6
:1016400010928500109284002BC02091BE02332797
:1016500027FD30958091990290E02817390704F50D
:101660008091BE02992787FD9095FC01EE0FFF1F28
:10167000E80FF91FE656FD4F808186FF11C080916B
:10168000BE02992787FD9095FC01EE0FFF1FE80F22
:10169000F91FE656FD4F80818F7360E00E94650D53
:1016A0008091BE028F5F8093BE022091BE023327DD
:1016B00027FD30958091990290E0281739070CF0AA
:1016C0004EC08091BE028C300CF049C02091840045
:1016D000309185008091BE02992787FD9095FC018D
:1016E000EE0FFF1FE80FF91FE656FD4F8181928133
:1016F000280F391F30938900209388008091BE0203
:10170000992787FD9095FC01EE0FFF1FE80FF91F49
:10171000E656FD4F808186FF2BC08091BE0299273F
:1017200087FD9095FC01EE0FFF1FE80FF91FE656AD
:10173000FD4F80818F7361E00E94650D19C080E4C8
:101740009CE905C080918400909185000496909357
:101750008900809388008FEF8093BE0209C080913A
:10176000840090918500049680549C4940F3EACF10
:10177000FF91EF91BF91AF919F918F917F916F9169
:101780005F914F913F912F910F900FBE0F901F903F
:101790001895F999FECF72BD61BDF89A80B508958C
:1017A000F999FECF1FBA72BD61BD40BD0FB6F89466
:1017B000FA9AF99A0FBE08951F920F920FB60F92E0
:1017C00011242F933F938F939F93AF93BF93809157
:1017D000C4029091C502A091C602B091C702309197
:1017E000C8020196A11DB11D232F2D5F2D3720F0BA
:1017F0002D570196A11DB11D2093C8028093C402EC
:101800009093C502A093C602B093C7028091C00214
:101810009091C102A091C202B091C3020196A11D94
:10182000B11D8093C0029093C102A093C202B093F5
:10183000C302BF91AF919F918F913F912F910F90D4
:101840000FBE0F901F9018958FB7F8942091C40287
:101850003091C5024091C6025091C7028FBFB901B5
:10186000CA0108959B01AC017FB7F8948091C00232
:101870009091C102A091C202B091C30266B5A89B2B
:1018800005C06F3F19F00196A11DB11D7FBFBA2F92
:10189000A92F982F8827860F911DA11DB11D62E0E9
:1018A000880F991FAA1FBB1F6A95D1F7BC012DC0D5
:1018B000FFB7F8948091C0029091C102A091C2023A
:1018C000B091C302E6B5A89B05C0EF3F19F00196A1
:1018D000A11DB11DFFBFBA2FA92F982F88278E0FEA
:1018E000911DA11DB11DE2E0880F991FAA1FBB1F0A
:1018F000EA95D1F7861B970B885E9340C8F221507A
:1019000030404040504068517C4F21153105410521
:10191000510571F60895789484B5826084BD84B5CC
:10192000816084BD85B5826085BD85B5816085BDDA
:10193000EEE6F0E0808181608083E1E8F0E01082F3
:10194000808182608083808181608083E0E8F0E034
:10195000808181608083E1EBF0E08081846080831E
:10196000E0EBF0E0808181608083EAE7F0E0808155
:1019700084608083808182608083808181608083B5
:101980008081806880831092C10008951F93CF9357
:10199000DF93182FEB0161E00E94260D209709F4D8
:1019A0004AC0CF3FD10509F449C0E12FF0E0E2552C
:1019B000FF4F84918330C1F0843028F4813051F09E
:1019C0008230B1F50CC0863019F1873049F184308E
:1019D00079F514C084B5806884BDC7BD33C084B5B3
:1019E000806284BDC8BD2EC08091800080688093D5
:1019F0008000D0938900C093880024C0809180002B
:101A0000806280938000D0938B00C0938A001AC0BC
:101A10008091B00080688093B000C093B30012C082
:101A20008091B00080628093B000C093B4000AC07F
:101A3000C038D1051CF4812F60E002C0812F61E025
:101A40000E94650DDF91CF911F910895CF93DF9391
:101A5000482F50E0CA0186569F4FFC0134914A57E7
:101A60005F4FFA018491882369F190E0880F991FF4
:101A7000FC01E859FF4FA591B491FC01EE58FF4FCE
:101A8000C591D491662351F42FB7F8948C91932F7C
:101A9000909589238C93888189230BC0623061F4EF
:101AA0002FB7F8948C91932F909589238C938881EC
:101AB000832B88832FBF06C09FB7F8948C91832B0C
:101AC0008C939FBFDF91CF910895482F50E0CA01BA
:101AD00082559F4FFC012491CA0186569F4FFC01FD
:101AE00094914A575F4FFA013491332309F440C06F
:101AF000222351F1233071F0243028F42130A1F059
:101B0000223011F514C02630B1F02730C1F0243056
:101B1000D9F404C0809180008F7703C08091800049
:101B20008F7D8093800010C084B58F7702C084B50C
:101B30008F7D84BD09C08091B0008F7703C08091F4
:101B4000B0008F7D8093B000E32FF0E0EE0FFF1F19
:101B5000EE58FF4FA591B4912FB7F894662321F466
:101B60008C919095892302C08C91892B8C932FBFE7
:101B70000895682F70E0CB0182559F4FFC0124919E
:101B8000CB0186569F4FFC0144916A577F4FFB0162
:101B90009491992319F420E030E03CC0222351F1C4
:101BA000233071F0243028F42130A1F0223011F5D7
:101BB00014C02630B1F02730C1F02430D9F404C06D
:101BC000809180008F7703C0809180008F7D80930B
:101BD000800010C084B58F7702C084B58F7D84BD2E
:101BE00009C08091B0008F7703C08091B0008F7DD5
:101BF0008093B000892F90E0880F991F84589F4FE1
:101C0000FC01A591B4918C9120E030E0842311F087
:101C100021E030E0C9010895CF93DF930E948B0C3F
:101C20000E944106C7E5DEE00E94A0042097E1F390
:101C30000E94570EF9CF08951F920F920FB60F9280
:101C400011242F933F934F938F939F93EF93FF9381
:101C50008091C00082FD1DC04091C6002091090303
:101C600030910A032F5F3F4F2F73307080910B0329
:101C700090910C032817390771F0E0910903F09156
:101C80000A03E753FD4F408330930A03209309036F
:101C900002C08091C600FF91EF919F918F914F916B
:101CA0003F912F910F900FBE0F901F901895E091CC
:101CB0005D03F0915E03E05CFF4F81919191208183
:101CC0003181821B930B8F739070892B11F00E94CE
:101CD0001B0E08951F920F920FB60F9211242F938F
:101CE0003F938F939F93EF93FF9320914D033091F8
:101CF0004E0380914F03909150032817390731F418
:101D00008091C1008F7D8093C10014C0E0914F038A
:101D1000F0915003E35FFC4F208180914F0390913D
:101D2000500301968F7390709093500380934F03EC
:101D30002093C600FF91EF919F918F913F912F913A
:101D40000F900FBE0F901F901895AF92BF92DF9229
:101D5000EF92FF920F931F93CF93DF93EC017A01E1
:101D60008B01DD24403081EE580780E0680780E079
:101D7000780711F0DD24D39491E0A92EB12CEC89E1
:101D8000FD89DD2069F0C50108A002C0880F991FF8
:101D90000A94E2F7808360E079E08DE390E005C08B
:101DA000108260E874E88EE190E0A80197010E943B
:101DB000FB14215030404040504056954795379590
:101DC000279580E12030380720F0DD2011F0DD2458
:101DD000D6CFE889F9893083EA89FB89208319A263
:101DE000EE89FF89408121E030E0C9010C8C02C0FE
:101DF000880F991F0A94E2F7482B4083EE89FF89E8
:101E00004081C9010D8C02C0880F991F0A94E2F726
:101E1000482B4083EE89FF894081C9010E8C02C0A6
:101E2000880F991F0A94E2F7482B4083EE89FF89B7
:101E300080810F8C02C0220F331F0A94E2F7209595
:101E400028232083DF91CF911F910F91FF90EF9076
:101E5000DF90BF90AF900895DC011C96ED91FC914E
:101E60001D97E05CFF4F2191319180819181281B6A
:101E7000390B2F733070C9010895DC011C96ED9168
:101E8000FC911D97E05CFF4F20813181E054F040D0
:101E9000DF01AE5BBF4F8D919C91119728173907D9
:101EA00019F42FEF3FEF07C08D919C91E80FF91FB8
:101EB0008081282F30E0C9010895DC011C96ED9146
:101EC000FC911D97E05CFF4F20813181E054F04090
:101ED000DF01AE5BBF4F8D919C9111972817390799
:101EE00019F42FEF3FEF10C08D919C911197E80FDF
:101EF000F91F20818D919C91119701968F7390709D
:101F000011969C938E9330E0C9010895DC0191965F
:101F10008C919197882339F05496ED91FC915597C7
:101F2000808186FFF9CF91961C920895CF93DF931D
:101F3000EC01EE85FF85E05CFF4F20813181E054AC
:101F4000F0402F5F3F4F2F733070DF01AE5BBF4F0C
:101F50008D919C91119728173907D1F3E05CFF4FC1
:101F600080819181E054F040E80FF91F6083EE8595
:101F7000FF85E05CFF4F31832083EE89FF8920815C
:101F800081E090E00F8C02C0880F991F0A94E2F75D
:101F9000282B208381E089A3EC89FD8980818064DE
:101FA000808381E090E0DF91CF91089510925403F7
:101FB0001092530388EE93E0A0E0B0E080935503C5
:101FC00090935603A0935703B09358038BE791E087
:101FD000909352038093510389EC92E090935E03B7
:101FE00080935D038DE093E09093600380935F03A3
:101FF00085EC90E0909362038093610384EC90E021
:10200000909364038093630380EC90E09093660365
:102010008093650381EC90E090936803809367035D
:1020200082EC90E090936A038093690386EC90E0E1
:1020300090936C0380936B0384E080936D0383E043
:1020400080936E0387E080936F0385E08093700335
:1020500081E08093710308952F923F924F925F9297
:102060006F927F928F929F92AF92BF92CF92DF92A8
:10207000EF92FF920F931F93DF93CF93CDB7DEB70D
:102080003B014C0119012A016D897E898F89988D48
:102090006A197B098C099D09621A730A840A950AD8
:1020A000A40193010E94BD14E218F3080409150964
:1020B000A80197010E941D152A0D3B1D4C1D5D1D99
:1020C000B901CA01CF91DF911F910F91FF90EF905D
:1020D000DF90CF90BF90AF909F908F907F906F9048
:1020E0005F904F903F902F900895CF92DF92EF92A4
:1020F000FF920F931F93CF93DF937C016B018A01B3
:10210000C0E0D0E00FC0D6016D916D01D701ED9117
:10211000FC910190F081E02DC7010995C80FD91FEE
:10212000015010400115110571F7CE01DF91CF91DB
:102130001F910F91FF90EF90DF90CF900895EF9255
:10214000FF920F931F938C01DC01ED91FC910190A4
:10215000F081E02D6DE009957C01D801ED91FC91B5
:102160000190F081E02DC8016AE009959C012E0DD7
:102170003F1DC9011F910F91FF90EF900895CF93DC
:10218000DF93EC016115710519F420E030E00FC018
:10219000DB010D900020E9F71197A61BB70BE88132
:1021A000F9810280F381E02DAD0109959C01C901FF
:1021B000DF91CF9108954F925F927F928F929F927D
:1021C000AF92BF92CF92DF92EF92FF920F931F9345
:1021D000DF93CF93CDB7DEB7A1970FB6F894DEBFEC
:1021E0000FBECDBF2C01742ECB01223008F42AE0A3
:1021F00019A231E2C32ED12CCC0EDD1E822E9924E1
:10220000AA24BB24672D752FA50194010E94FB14FD
:1022100079018A01C801B701A50194010E94BD148A
:10222000472D461B0894C108D1084A3014F4405D7C
:1022300001C0495CF6014083E114F1040105110578
:1022400021F07E2C5F2DC801DDCFC201B6010E94B6
:10225000BF10A1960FB6F894DEBF0FBECDBFCF91D1
:10226000DF911F910F91FF90EF90DF90CF90BF9083
:10227000AF909F908F907F905F904F900895DC017A
:102280002115310541F4ED91FC910190F081E02D93
:10229000642F099508950E94DB100895CF92DF9274
:1022A000EF92FF920F931F93CF93DF93EC016A019C
:1022B0007B012115310541F4E881F9810190F0811C
:1022C000E02D642F09951FC02A303105D1F477FF26
:1022D00017C0E881F9810190F081E02D6DE2099548
:1022E0008C0144275527BA014C195D096E097F09F5
:1022F000CE012AE00E94DB109801280F391F04C08C
:102300002AE00E94DB109C01C901DF91CF911F914F
:102310000F91FF90EF90DF90CF900895EF92FF9292
:102320000F931F937B019A010027F7FC0095102F54
:10233000B801A7010E944E111F910F91FF90EF90DD
:1023400008950E94BF1008957F928F929F92AF923E
:10235000BF92CF92DF92EF92FF920F931F93CF9392
:10236000DF934C017A018B01722ECB01BA01A801D7
:1023700097010E94B914882321F0C40168E671E036
:1023800021C0C0E0D0E057016801E894D7F8C60149
:10239000B5012FEF3FEF4FE75FE70E94B9148823A5
:1023A00051F4C601B5012FEF3FEF4FE75FE70E9401
:1023B0000313181614F0C1E0D0E0219739F0C401DE
:1023C0006CE671E00E94BF10EC0193C0C801B70138
:1023D0002FEF3FEF4FE75FE40E945214181654F0BE
:1023E000C801B7012FEF3FEF4FE75FEC0E940313E7
:1023F000882324F4C40160E771E0E4CFC801B70189
:1024000020E030E040E050E00E94031387FD03C06D
:10241000C0E0D0E00EC0D401ED91FC910190F081BC
:10242000E02DC4016DE20995EC0117FB109517F939
:10243000109520E030E040E05FE3DD240BC0CA01EE
:10244000B90120E030E040E251E40E9407139B0113
:10245000AC01D394D71498F3C801B7010E949F121E
:102460005B016C010E9474137B018C01C401B801F3
:10247000A7012AE030E00E943F11C80FD91F772042
:1024800039F0C40164E771E00E94BF10C80FD91F82
:10249000C801B7010E94A0139B01AC01C601B501A0
:1024A0000E949E1224C020E030E040E251E40E94ED
:1024B00056147B018C010E946F135B016C01CC24CC
:1024C000B7FCC094DC2CC401B601A5012AE030E0C1
:1024D0000E944E11C80FD91FC601B5010E94A21358
:1024E0009B01AC01C801B7010E949E127A9477202B
:1024F000D1F6CE01DF91CF911F910F91FF90EF9018
:10250000DF90CF90BF90AF909F908F907F90089575
:102510000E94A4110895EF92FF920F931F937C01E4
:102520000E94BF108C01C7010E949F10080F191F45
:10253000C8011F910F91FF90EF9008955058BB274D
:10254000AA270ED075C166D130F06BD120F031F4DE
:102550009F3F11F41EF45BC10EF4E095E7FB51C1FF
:10256000E92F77D180F3BA176207730784079507BD
:1025700018F071F49EF58FC10EF4E0950B2EBA2F72
:10258000A02D0B01B90190010C01CA01A001112479
:10259000FF27591B99F0593F50F4503E68F11A1625
:1025A000F040A22F232F342F4427585FF3CF4695B6
:1025B00037952795A795F0405395C9F77EF41F16D8
:1025C000BA0B620B730B840BBAF09150A1F0FF0FA2
:1025D000BB1F661F771F881FC2F70EC0BA0F621F8E
:1025E000731F841F48F4879577956795B795F7957E
:1025F0009E3F08F0B3CF9395880F08F09927EE0F10
:10260000979587950895D9D008F481E008950CD066
:102610000FC107D140F0FED030F021F45F3F19F038
:10262000F0C0511139C1F3C014D198F39923C9F303
:102630005523B1F3951B550BBB27AA2762177307C8
:10264000840738F09F5F5F4F220F331F441FAA1F7C
:10265000A9F333D00E2E3AF0E0E830D0915050403C
:10266000E695001CCAF729D0FE2F27D0660F771FEA
:10267000881FBB1F261737074807AB07B0E809F0CC
:10268000BB0B802DBF01FF2793585F4F2AF09E3F61
:10269000510568F0B6C000C15F3FECF3983EDCF333
:1026A000869577956795B795F7959F5FC9F7880FDA
:1026B000911D9695879597F90895E1E0660F771F2C
:1026C000881FBB1F621773078407BA0720F0621BBD
:1026D000730B840BBA0BEE1F88F7E095089504D0B6
:1026E0006894B111D9C00895BCD088F09F5790F07C
:1026F000B92F9927B751A0F0D1F0660F771F881F27
:10270000991F1AF0BA95C9F712C0B13081F0C3D041
:10271000B1E00895C0C0672F782F8827B85F39F0DF
:10272000B93FCCF3869577956795B395D9F73EF485
:1027300090958095709561957F4F8F4F9F4F08952D
:10274000E89409C097FB3EF490958095709561954B
:102750007F4F8F4F9F4F9923A9F0F92F96E9BB2701
:102760009395F695879577956795B795F111F8CF7D
:10277000FAF4BB0F11F460FF1BC06F5F7F4F8F4FE8
:102780009F4F16C0882311F096E911C0772321F0DE
:102790009EE8872F762F05C0662371F096E8862F76
:1027A00070E060E02AF09A95660F771F881FDAF7CD
:1027B000880F9695879597F90895990F0008550FFA
:1027C000AA0BE0E8FEEF16161706E807F907C0F0B7
:1027D00012161306E407F50798F0621B730B840BBF
:1027E000950B39F40A2661F0232B242B252B21F499
:1027F00008950A2609F4A140A6958FEF811D811D39
:10280000089597F99F6780E870E060E008959FEF72
:1028100080EC089500240A94161617061806090677
:10282000089500240A941216130614060506089546
:10283000092E0394000C11F4882352F0BB0F40F4CE
:10284000BF2B11F460FF04C06F5F7F4F8F4F9F4F0E
:10285000089557FD9058440F551F59F05F3F71F090
:102860004795880F97FB991F61F09F3F79F08795F7
:102870000895121613061406551FF2CF4695F1DF80
:1028800008C0161617061806991FF1CF8695710510
:10289000610508940895E894BB2766277727CB0144
:1028A00097F908958ADF08F48FEF08950BD0C0CF11
:1028B000B1DF28F0B6DF18F0952309F0A2CFA7CF3B
:1028C0001124EACFC6DFA0F3959FD1F3950F50E016
:1028D000551F629FF001729FBB27F00DB11D639FD2
:1028E000AA27F00DB11DAA1F649F6627B00DA11D78
:1028F000661F829F2227B00DA11D621F739FB00D1E
:10290000A11D621F839FA00D611D221F749F33278D
:10291000A00D611D231F849F600D211D822F762F26
:102920006A2F11249F5750408AF0E1F088234AF023
:10293000EE0FFF1FBB1F661F771F881F915050406F
:10294000A9F79E3F510570F05CCFA6CF5F3FECF337
:10295000983EDCF3869577956795B795F795E7955B
:102960009F5FC1F7FE2B880F911D9695879597F96C
:10297000089523DF880B990B0895629FD001739F00
:10298000F001829FE00DF11D649FE00DF11D929F0B
:10299000F00D839FF00D749FF00D659FF00D99274A
:1029A000729FB00DE11DF91F639FB00DE11DF91F6E
:1029B000BD01CF0111240895991B79E004C0991F2E
:1029C000961708F0961B881F7A95C9F78095089589
:1029D00097FB092E07260AD077FD04D049D006D0F0
:1029E00000201AF4709561957F4F0895F6F7909541
:1029F00081959F4F0895A1E21A2EAA1BBB1BFD01D2
:102A00000DC0AA1FBB1FEE1FFF1FA217B307E407CD
:102A1000F50720F0A21BB30BE40BF50B661F771F25
:102A2000881F991F1A9469F7609570958095909505
:102A30009B01AC01BD01CF01089597FB092E05262E
:102A40000ED057FD04D0D7DF0AD0001C38F45095C3
:102A50004095309521953F4F4F4F5F4F0895F6F7C2
:102A600090958095709561957F4F8F4F9F4F0895FA
:102A7000AA1BBB1B51E107C0AA1FBB1FA617B707A4
:102A800010F0A61BB70B881F991F5A95A9F78095C0
:102A90009095BC01CD010895EE0FFF1F0590F491B4
:082AA000E02D0994F894FFCF2A
:102AA8003C76657273696F6E3A302E3132373E006C
:102AB8003C6D6F766564200020003E003C73746FA7
:102AC800703E003C69643A3A6D616C673E00003CB8
:102AD800656570726F6D206572617365643E003C58
:102AE800686F72697A5F656570726F6D3A20003C35
:102AF80073746F706465746563746661696C3E00B5
:102B08003C72657365743E006E616E00696E6600A6
:102B18006F7666002E000100000000960F75102CDD
:082B28000F5D0F3D0F860F0049
:00000001FF
